:020000040000FA
:10000000B4017929A400380884003608DD2084135F
:1000100000052C1C3606031920282408031D182867
:100020002A08FF3E031C21283230F1202A0821280B
:10003000240AFF3003192028240B20282B0821280C
:10004000AD09AD0C7429B416B41EB41234192D28A0
:10005000FE39B500341503107429341A3528A6006A
:1000600034164C2003183A282608532003183A283F
:10007000B41E742945206A2034113412B411380892
:1000800084003608841780044B2838088400360919
:1000900080058417800508003F206A2045206620DF
:1000A0003508B4190138A2000830A300A20D0318C6
:1000B0003F20031C45206A206620A30B56283F20C2
:1000C0006A203808840036080005FF3E390884009D
:1000D000370948283908840037084228A501A400B8
:1000E000B5172730A300103081200330A300E8307B
:1000F0008120A30164308120A3010A3081202408DB
:100100008C28A2002508A1002408A0004221200874
:10011000031DB513B51B0800303EA700851305135A
:1001200005138316851305130513F0308505831217
:100130002708B418B9283A30A1009830FF2033308E
:10014000A600CE201330A1008830FF20CE206430DE
:10015000FE20CE206430FE202230A600CE202830A3
:10016000B8200C30B8200630B820B4142708B928BD
:100170003414A600341CC7280513033C031CCC28E8
:10018000CC200730A100D030FF2003140800341425
:10019000FE3C031974290517A60E341C341085176C
:1001A000F030850526080F3985048513A60E34180E
:1001B000CE283230FE2003140800841780047429EE
:1001C00083169B001C141A08742983169A001C15A8
:1001D00055309D00AA309D009C149C18ED281C11E0
:1001E0007429A301A200FF30A207031CA307031C6C
:1001F00074290330A100DF30FF20F328A101E83E7D
:10020000A000A109FC30031C0829A0070318052938
:10021000A0076400A10F052920180E29A01C12298F
:100220000000122908000310A00DA10DFF3E0318C5
:10023000132920087429A20003302429A2000630C3
:100240002429A20004302429A80023082102031D28
:100250002B29220820020430031801300319023030
:100260002805031DFF307429A2002008A6002408D9
:10027000A0002608A4002108A6002508A100260841
:10028000A5004429A501A4011030A600210DA40D4C
:10029000A50D2208A4022308031C230FA50203189E
:1002A00058292208A40723080318230FA5070310C1
:1002B000A00DA10DA60B4629200874291030A80016
:1002C000A101A001A70CA60C031C6C292208A00701
:1002D00023080318230FA107A10CA00CA50CA40C44
:1002E000A80B622924087429831303138312640062
:1002F00008008316061506148615831207309F0022
:10030000831681018312C030C6000130D200013053
:10031000D0000130CF006430F1202F2231308D2009
:100320004D308D2046308D204B308D202D308D204E
:1003300050308D204C308D204C308D20FE308D2063
:10034000C0308D2053308D2044308D2041308D20A1
:1003500033308D2033308D2030308D2032308D2061
:1003600065308D200730A300D030F2200030E0202F
:10037000C4000130E020C5000230E020D30003308B
:10038000E020CD000430E020CE0061220630B8002D
:100390000230B6000630B9001030B70046082520FC
:1003A00045082520440823207322AC220630B800DB
:1003B0000430B600AC01FE30AA00C830AB000130FA
:1003C000AD0048080220C8000318082A0630B8000B
:1003D0000130B600AC01FE30AA00C830AB000130DD
:1003E000AD0049080220C90003181B2A0630B800D6
:1003F0000830B600AC01FF30AA00AB010130AD00FF
:100400004A080220CA000318192BC830FE20D6293A
:100410005208C4070318C50A4408A0004508A100F3
:100420005730A30080302121031D1A2AA030C400B8
:100430000F30C500FB2A4408A0004508A1000F307A
:10044000A300A0301E21031D2A2A5208C402031C47
:10045000C503FB2A8030C4005730C500FB2AFE309C
:100460008D2001308D200800FE308D20C0308D2081
:10047000080043308D2074308D2072308D206C3018
:100480008D2062308D2079308D2074308D200800D1
:1004900045308D2058308D2049308D2054308D20AE
:1004A0000800342276308D20FE308D20C2308D2021
:1004B0005E308D20FE308D20C7308D207E308D2027
:1004C00008000630B8000230B6000630B90010301F
:1004D000B700460825204D0825204E082320080097
:1004E0000130CF00192B7D30A600A7015308A200D0
:1004F000A3015E21BC002508BD004408A6004508F4
:10050000A7003C08A2003D08A3005E21BA00250810
:10051000BB000730A300D0303421C0002108C10047
:100520004408A6004508A7005308A200A3015E21C5
:10053000C2002508C3000F30C2050030C3054208C1
:10054000A6004308A7007130A2000230A3005E217C
:10055000BE002508BF0008002F224008A000410867
:10056000A1002730A30010301B21031DC52A203015
:100570008D204008A0004108A1000330A300E8300E
:100580001B21031DC52A20308D204108A5004008ED
:100590006F202E308D2034223E08A0003F08A1009D
:1005A0000330A300E8301B21031DEE2A30308D20DC
:1005B0003E08A0003F08A100A30164301B21031DD9
:1005C000EE2A30308D203E08A0003F08A100A30194
:1005D0000A301B21031DEE2A30308D203F08A50074
:1005E0003E086F2020308D204D308D2048308D20EA
:1005F0007A308D20080083169B0183124408E52081
:10060000831601309B0083124508E52083160230D3
:100610009B0083125308E520831603309B0083124E
:100620004D08E520831604309B0083124E08E52018
:10063000C6292F2264005008013C031D2E2B533085
:100640008D2063308D2068308D2072308D20693090
:100650008D2074308D2074308D20672B64005008FD
:10066000023C031D402B46308D2061308D206B30C5
:100670008D2074308D206F308D2072308D20672B4F
:1006800064005008033C031D492B392231308D2072
:10069000672B64005008043C031D522B3922323072
:1006A0008D20672B64005008053C031D672B4630E6
:1006B0008D2072308D2065308D2071308D20753009
:1006C0008D2065308D206E308D207A308D20512226
:1006D0000630B8000430B600AC01FF30AA00AB0110
:1006E0000130AD0048080220C8000318962B0630E0
:1006F000B8000130B600AC01FF30AA00AB010130F8
:10070000AD0049080220C90003189F2B0630B8002D
:100710000830B600AC01FF30AA00AB010130AD00DB
:100720004A080220CA000318A82B682BD00A6400CC
:1007300006305002031C9E2B0130D000192BD00331
:100740006400013050020318A72B0530D000192B8C
:1007500064005008013C0319212C64005008023C3D
:100760000319C12B64005008033C0319BF2C64001B
:100770005008043C03196A2D64005008053C031915
:10078000FB2A2F2246308D2061308D206B308D204A
:1007900074308D206F308D2072308D2034225308BC
:1007A0006E202D308D2066308D2061308D2063309D
:1007B0008D2068308D200630B8000430B600AC01C2
:1007C000FF30AA00AB010130AD0048080220C8008C
:1007D0000318092C0630B8000130B600AC01FF3018
:1007E000AA00AB010130AD0049080220C90003187E
:1007F000122C0630B8000830B600AC01FF30AA0059
:10080000AB010130AD004A080220CA000318192BC1
:10081000DB2BD30A64000B305302031C112C013074
:10082000D3001A2CD30364000130530203181A2C8E
:100830000A30D300831602309B0083125308E52050
:10084000C12B2F2253308D2063308D2068308D20B6
:1008500072308D2069308D2074308D2074308D2061
:100860003A308D2034227130A6000230A7005208A1
:10087000A200A3015E21B2002508B3003208A60041
:100880003308A7005308A200A3015E21C200250877
:10089000C3004208A0004308A1000A30A200A3013F
:1008A0004221C0002108C1004108A50040086F2076
:1008B0002E308D2001304205BE0000304305BF00C0
:1008C0003E08A6003F08A7000530A200A3015E2154
:1008D000B2002508B3003308A50032086F206B3042
:1008E0008D2048308D207A308D200630B8000430BD
:1008F000B600AC01FF30AA00AB010130AD004808E2
:100900000220C8000318A32C0630B8000130B6003E
:10091000AC01FF30AA00AB010130AD004908022054
:10092000C9000318B42C0630B8000830B600AC017A
:10093000FF30AA00AB010130AD004A080220CA0016
:100940000318192B752C640010305202031CAB2CB9
:100950000130D200B32C5208A600A7010230A20039
:10096000A3015E21D200212C640002305202031840
:10097000BC2C1030D200BE2C0310D20C212C2F2204
:1009800064004F08073C031DCA2C35308D204930C8
:100990008D20EE2C64004F08053C031DD42C5430F0
:1009A0008D2030308D20EE2C64004F08063C031D56
:1009B000DE2C54308D2031308D20EE2C64004F0819
:1009C000013C031DE82C4F308D2053308D20EE2C40
:1009D00064004F08083C031DEE2C482264004F08B9
:1009E000083C0319152D0130CB00FF304F07B20032
:1009F000FF300318013EB3004B08A000A1013208EC
:100A00001621CB004D084B05CC0020308D203D3009
:100A10008D2020308D2064004C08003C031D132DD8
:100A200030308D20152D31308D2051220630B80008
:100A30000430B600AC01FF30AA00AB010130AD00BC
:100A400048080220C8000318442D0630B8000130C1
:100A5000B600AC01FF30AA00AB010130AD0049087F
:100A60000220C9000318542D0630B8000830B60023
:100A7000AC01FF30AA00AB010130AD004A080220F2
:100A8000CA000318642D162DCF0A64004F08023CDB
:100A9000031D4C2D0530CF00640009304F02031CAC
:100AA000532D0130CF00BF2CCF0364004F08043C0E
:100AB000031D5C2D0130CF00640001304F0203188C
:100AC000632D0830CF00BF2C64004F08083C031D85
:100AD000762E702A2F2250308D20FF304F07B20023
:100AE000FF300318013EB3003308A50032086F2021
:100AF0000130CB00FF304F07B200FF300318013E3A
:100B0000B3004B08A000A10132081621CB004E080B
:100B10004B05CC0020308D203D308D2020308D20A5
:100B200064004C08003C031D9A2D41308D206E302E
:100B30008D20A02D41308D2075308D2073308D207B
:100B400064004F08093C031DA72D2F224822512283
:100B50000630B8000430B600AC01FF30AA00AB018B
:100B60000130AD0048080220C8000318D62D063019
:100B7000B8000130B600AC01FF30AA00AB01013073
:100B8000AD0049080220C9000318E62D0630B80060
:100B90000830B600AC01FF30AA00AB010130AD0057
:100BA0004A080220CA000318F62DA82DCF0A6400B7
:100BB0000A304F02031CDE2D0130CF0064004F08C5
:100BC000043C031DE52D0530CF006A2DCF036400E2
:100BD00001304F020318EE2D0930CF0064004F089A
:100BE000043C031DF52D0330CF006A2D64004F082F
:100BF000093C031DFC2D702A2F2250308D206F30B0
:100C00008D2072308D2074308D20FF304F07B20060
:100C1000FF300318013EB3003308A50032086F20EF
:100C20003D308D2034220130CB00FF304F07B20021
:100C3000FF300318013EB3004B08A000A1013208A9
:100C40001621CB004E084B05CC0064004C08003C3C
:100C5000031D2F2E41308D206E308D20352E4130DA
:100C60008D2075308D2073308D200630B800043013
:100C7000B600AC01FF30AA00AB010130AD0048085E
:100C80000220C8000318632E0630B8000130B600F9
:100C9000AC01FF30AA00AB010130AD0049080220D1
:100CA000C9000318632E0630B8000830B600AC0146
:100CB000FF30AA00AB010130AD004A080220CA0093
:100CC00003186A2D352E0130CB00FF304F07B200DC
:100CD000FF300318013EB3004B08A000A101320809
:100CE0001621CB004B08CE066122FC2D2F2264007A
:100CF0004F08073C031D812E35308D2049308D2053
:100D00009E2E64004F08053C031D8B2E54308D2011
:100D100030308D209E2E64004F08063C031D952E1A
:100D200054308D2031308D209E2E64004F08013CC0
:100D3000031D9E2E4F308D2053308D203D308D2051
:100D400034220130CB00FF304F07B200FF300318D0
:100D5000013EB3004B08A000A10132081621CB00D0
:100D60004D084B05CC0064004C08003C031DBB2E15
:100D700030308D20BD2E31308D200630B80004304B
:100D8000B600AC01FF30AA00AB010130AD0048084D
:100D90000220C8000318EB2E0630B8000130B60060
:100DA000AC01FF30AA00AB010130AD0049080220C0
:100DB000C9000318EB2E0630B8000830B600AC01AD
:100DC000FF30AA00AB010130AD004A080220CA0082
:100DD0000318BF2CBD2E0130CB00FF304F07B200EF
:100DE000FF300318013EB3004B08A000A1013208F8
:0C0DF0001621CB004B08CD066122762EA8
:02400E00703F01
:0A420000000050000100CE00000095
:00000001FF
